:020000040000FA
:06000000FE300F306A28FB
:08000800A000030EA100831209
:10001000C31D3B288B1C34288B1031181628B11CAB
:10002000342864300102031833281A2800001828E5
:1000300019281A281B281C281D281E281F2820289C
:1000400021283110B114A810031005190314AA0DAA
:10005000A90DA80DB00B342831152A08AF002908C6
:10006000AE002808AD00B11081010B11210E8300F4
:10007000A00E200E090005194328831601178312CC
:10008000B23081005E2883160113831203140B190A
:100090000310A80DA90DAA0DAB0DAC0DAC16FF30C9
:1000A0002C02031D5E28FA302B02031D5E28311539
:1000B0002A08AF002908AE002808AD008B100B11EC
:0A00C000210E8300A00E200E09009F
:0C00D400203084008001840A8030040287
:1000E000031C6C281230B0005A30C000C10001302F
:1000F000D400D500E400E500E300F100F000EE00DC
:100100000730D8008030D7001F30E6000717FA30DC
:10011000FD000330EF0083160F3085052030860583
:100120000D30870583128501860187011030831603
:100130008E008312703083168F00831200300317F5
:1001400099000313003003179A000313003097003F
:1001500000309F00003083169F0083120030031789
:100160009E000313003003179F000313C030831653
:1001700081008312313090000030920000308316ED
:100180009400831200309400A630831698008312E6
:10019000003083169B008312903098003330831612
:1001A00099008312003083168C008312003083166E
:1001B0008D00831210308B000D16692581018E0190
:1001C0008F010B118B100B108C128C018D010D16F1
:1001D0008B1713235123792124213119DB23311A61
:1001E0003E21591CF622591887228F080319EC2842
:1001F0008F01C9228723FE21D0219021B021072918
:10020000E71BEB01EB0B0729E801E901EA01E71322
:100210005918EC28B1191929D60BEC28B11A0A3053
:10022000B11EC830D600B11A20297921CC0ACC19C8
:100230004A14B111B11A0A30B11EC830D600EC28E8
:100240007921BE186925EC286400C31DB113C31DB4
:100250000800311808000B1D08000B11B1103114F3
:100260001230B000051D3929B1178316011383120E
:100270000800B113831601178312080031124A10C7
:10028000CC0121305B02031D4B295C08CE005D08C8
:10029000CF00661774295B085C065D02031D080029
:1002A00077305B02031D58295C087406C40074296A
:1002B00066305B02031D5F295C08CB007429553052
:1002C0005B02031D66295C08F800742944305B0258
:1002D000031D6D295C08FA00742933305B02031D8D
:1002E00074295C08FB007429B116B1110A30D600DC
:1002F0000800591459158B138316071283128B1794
:10030000071608005910D9101930DE00B112B111CA
:10031000C830D6008B138316071683128B1708007C
:10032000051897291930C00703189C2908000A30BE
:10033000C002031CA8290800FF30C000421464302A
:100340004102031808004210C2144317C3140800E6
:10035000C0014210C213C21C0800C20143130800AE
:100360008518B7291930C1070318BC2908000A30BD
:10037000C102031CC8290800FF30C10042146430C8
:10038000400203180800421042154317C31008002A
:10039000C1014210C213421D0800C20143130800EC
:1003A000E303031D0800E0080319E329651860084A
:1003B000E51861086519620899000330E30003102D
:1003C000E50DE51D08001430E3000130E500EE08FE
:1003D0000319F529EE030319F3296030E605031D1F
:1003E000F529E00108001F30E6040310E40D0318AE
:1003F0006414640866050319F529132B8C1E080084
:10040000E7174A150717FA30FD001819CA146908CA
:10041000E8006A08E9001A08EA00E81F080068080E
:10042000C13C031D1B2A69086A05C3046A096904E3
:10043000C305C424862A6808C23C031D272A69080C
:100440006A05C5046A096904C505CA24862A6808BC
:10045000C43C031D2E2A6908F700862A6808FC3967
:10046000E03C031D3F2A690868188038BB006A0811
:10047000E8188038BA003C25BE143E14862A680865
:10048000FC39F03C031D5C2A690868188038EC00D0
:100490008B136C0803178D0083168C130C148312B6
:1004A0000C080313ED008B176C0334300319ED00B7
:1004B0003230EE00E616862A6808FC39803C031DBF
:1004C0006B2A690868188038CE006A08E8188038F6
:1004D000CF00D815862A6808FC39903C031D762A7F
:1004E000690868188038CE005816862A6808A03C2B
:1004F000031D862A69086A188038CD00C310EA18DF
:10050000C31445126A194516D816862A08005919C7
:10051000942AD3030F305305031D0800D308031991
:10052000972A0716D30E0800591B5D23591307128B
:100530005911D918822955185008D518510855193C
:1005400052085705031DA72AFF30D300AA2A2230DC
:10055000D300AA2A0310D70C0318AF2A0800803052
:10056000D7000310D50DD519B62A08000130D500E3
:100570000430D819D4000830581AD4000310D40D10
:1005800003185414540858050319B62A5123D914D2
:100590000800EF0B08000330EF00061EF42A0516D2
:1005A0000310F00D031CE22A0130F0000310F10DDE
:1005B000711EE22A0130F100F0004408F300C31A72
:1005C000F317051271187308F1187208711977087A
:1005D000F11DED2A4B084A188038700506120319E0
:1005E0008516031D8512080006160800DA0A03198D
:1005F000D9165916071E5912D91D0F2B591A0F2B30
:10060000B1155A08283CD91A0310DD0DDC0DDB0D9D
:10061000DA01D912DE0B0F2B31161930DE00D91595
:10062000591ED9110800E001E101E201641F1F2BEE
:100630004830E0004E08E1004F08E2006613E41E77
:10064000282B4730E0006C08E1006D08E200E6125C
:10065000641E302B4130E0007A08E1007B08E200A4
:10066000E41D382B4C30E0007708E1007808E20008
:10067000641D402B4530E0004A08E1004B08E200D1
:10068000E41C482B4630E0004308E1004408E20047
:10069000641C502B5830E0005930E1005A30E20021
:1006A0000800D001D101D201541C5B2BF730D000DF
:1006B0004308D100832BD41C622BA130D0007708D3
:1006C000D100832B541D692BA230D0004508D100E6
:1006D000832BD41D732BC130D0004E08D1004F089E
:1006E000D200D8110800541E7B2BC230D0004E0817
:1006F000D1005812832BD41E0800A730D0004D081B
:10070000D100D812832B50085106D2000800311FA7
:100710008C2BFC0303193113071F912BFD030319C5
:100720000713031044180314B20DF03032020319FA
:10073000431307184311071C43150719C311071D5D
:10074000C31587194312871D43168710751CAA2BE2
:10075000C31A8714FE0B08004418D325441C8712C3
:100760004A1C87174A18CB25790AF71BF707771B0E
:10077000BD2B790A77020318F7007808F2000310FE
:10078000790C013E78020318F200C3120310790CB1
:10079000013E460778020318C31646087802031C78
:1007A000C3160310790C013E4602031C08007802B0
:1007B000031CC31208003111311B0800591808002E
:1007C0004A100717FA30FD00B7010430B8000C30AA
:1007D000370230300318B807C319B8178B1320300D
:1007E0003707380703178D0083168C130C148312F8
:1007F0000C080313A400A500C030A506103037076D
:10080000380703178D0083168C130C1483120C0801
:100810000313A300A6000230A606003037073807EE
:1008200003178D0083168C130C1483120C0803130A
:10083000A200A7000130A7068B17B11F252C2209A3
:100840000339A200A309A409A509C31D342C220859
:100850002D02031DBE2C23082E02031DBE2C2408CE
:100860002F02031D812C402C24082F02031DBE2CB7
:1008700023082E02031D812C22082D02031DBE2CED
:1008800000303702031D492C431808004314C424C8
:10089000080001303702031D592CFF30FC003117CE
:1008A000441CC314441C1F2544184313441C431701
:1008B000080002303702031D672CFF30FC0031179F
:1008C000441CC314441C2725441C43170800033050
:1008D0003702031D6E2C441CC31408003030370748
:1008E00038077F3903178D0083168C130C1483127D
:1008F0000C080313F7005917441CD024FF30FC00E8
:100900003117C31D882C25082F02031DBE2C902CE7
:1009100026082E02031DBE2C27082D02031DBE2C07
:1009200000303702031D992C431C08004310C424D7
:10093000080001303702031DA92CFF30FC003117DD
:10094000441CC310441C162544184313441C43176D
:10095000080002303702031DB72CFF30FC003117AE
:10096000441CC310441C2725441C431708000330B3
:100970003702031DBE2C441CC3100800B70A1C30EC
:10098000370203180800E52B2130BB004308BA00EA
:100990003C2508002330BB004508BA003C25080070
:1009A000771B0800431A142D0310790C013E7702BF
:1009B0000318F7000318D42C770878020319F22CD7
:1009C0000318EA2C78087702C3187902C318013E8D
:1009D000FF00F92C77087802C31C7902C31C013E82
:1009E000FF00F92C0310790C013EFF00F518F70702
:1009F0000C2D0310790C013EF518013E7F02031CFB
:100A00000C2D0310790C013EF707790A77020318C1
:100A1000F7000318052D0C2D770878024313031DEA
:100A20004317F518431708000C2D08005917C31079
:100A3000780AF700790A77020318F70008005917B7
:100A4000C3147803F700790AF71BF7070800591752
:100A50000310790C78077902031C362D0319362D03
:100A60000310790C013E7807F70008000310790C99
:100A7000013E7802F7000800FF010530DF000D128B
:100A80003B08831203178D00831203133A08831265
:100A900003178C00831603178C130C158B138B1BF9
:100AA0004E2D55308D00AA308D008C148B170C11F3
:100AB000831203136400DF03031D632D0530DF0081
:100AC000FF030319662D0D1E5A2D08000C118B17FC
:100AD0003C2D8B138B1B692D313003178D00831632
:100AE0008C130C1483120C080313F4008B1774106E
:100AF0008B13323003178D0083168C130C14831262
:100B00000C080313F5008B178B13333003178D007C
:100B100083168C130C1483120C080313F6008B1726
:100B20003E18AB2D8B13213003178D0083168C13C9
:100B30000C1483120C080313C3008B1743138B137D
:100B4000233003178D0083168C130C1483120C08AA
:100B50000313C5008B178B13203003178D008316EA
:100B60008C130C1483120C080313C6008B17460A4F
:100B70000319C6018B13303003178D0083168C13B5
:100B80000C1483120C08031307183030F900F90312
:100B9000BE103E1008000708803A870008000708CA
:100BA000403A870008000708203A87000800FF0045
:100BB000D325FF0BD82D08000708023A870008004C
:084000000F00000003000400A2
:02400E00CC03E1
:1042000000003400FF00FF00400042004400460070
:104210004200430040004100460047004400450082
:10422000FF00FF00FF00FF00F200F600FA00FE00B2
:10423000F000F200F400F600F800FA00FC00FE00C6
:10424000FF00FF00FF000000E500E500E500E500DD
:10425000E900E900E900E900E900E900E900E90016
:104260001800000001000000FF00FF00FF00FF0039
:104270000000010002000300040005000600070022
:104280004300420041004000470046004500440012
:104290004400450046004700400041004200430002
:1042A000F000F200F400F600F800FA00FC00FE0056
:1042B000F000F200F400F600F800FA00FC00FE0046
:1042C000ED00ED00ED00ED00ED00ED00ED00ED0086
:1042D000F100F100F100F100F100F100F100F10056
:1042E000080009000A000B000C000D000E000F0072
:1042F0001000110012001300140015001600170022
:10430000FF00FF00FF00FF000000000000000000B1
:104310000300030003000300030003000300030085
:10432000FF00FF00FF00FF00C800C800C800C80071
:10433000C800C800C800C800C800C800C800C8003D
:10434000FF00FF00FF00FF00C300F300CF00FF00ED
:104350000300C3003300F3000F00CF003F00FF0055
:10436000FF00FF00FF00FF00FF00FF00FF00FF0055
:10437000FF00FF00FF00FF00FF00FF00FF00FF0045
:10438000020002000200020002000200020002001D
:10439000000000000000000000000000000000001D
:1043A000C800C800C800C800C800C800C800C800CD
:1043B00088008800880088008800880088008800BD
:1043C0000300C3003300F3000F00CF003F00FF00E5
:1043D0000300C3003300F3000F00CF003F00FF00D5
:1043E000FF00FF00FF00FF00FF00FF00FF00FF00D5
:1043F000FF00FF00FF00FF00FF00FF00FF00FF00C5
:00000001FF
